:020000040800F2
:10000000001000205519000885040008910400081C
:1000100000000000000000000000000000000000E0
:10002000000000000000000000000000950400082F
:100030000000000000000000A1040008AD0400085A
:10004000A119000800000000A1190008A11900086A
:10005000A1190008A1190008A1190008A119000898
:100060000000000063070008A90A0008A1190008A1
:10007000A1190008A1190008A1190008000000003A
:10008000A11900080000000000000000A1190008EC
:1000900000000000C9030008A1190008A119000808
:1000A000000000009D03000800000000A1190008E6
:1000B0000000000000000000000000000000000040
:1000C00080B582B000AF0200FB1D1A70FB1D1B78CB
:1000D0001A001F231A40044B012191400A001A60A4
:1000E000C046BD4602B080BD00E100E090B583B0DF
:1000F00000AF02003960FB1D1A70FB1D1B787F2BBF
:1001000032D92F4AFB1D1B7819000F230B40083BE7
:100110009B0806339B00D31804331B68FA1D127822
:10012000110003220A40D200FF2191400A00D2436D
:100130001A4011003B689B01FF221A40FB1D1B78EF
:10014000180003230340DB009A401D48FB1D1B7869
:100150001C000F232340083B9B080A4306339B00E7
:10016000C31804331A6027E0164AFB1D1B785BB2E4
:100170009B08C0339B009B58FA1D12781100032284
:100180000A40D200FF2191400A00D2431A401100D8
:100190003B689B01FF221A40FB1D1B7818000323BC
:1001A0000340DB009A400748FB1D1B785BB29B08AD
:1001B0000A43C0339B001A50C046BD4603B090BDF1
:1001C00000ED00E000E100E080B582B000AF7860B3
:1001D0007B685A1E80235B049A4201D3012310E0FE
:1001E0000A4B7A68013A5A6001235B4203211800E6
:1001F000FFF77CFF054B00229A60044B07221A6030
:1002000000231800BD4602B080BDC04610E000E0EB
:1002100080B500AFC046BD4680BD80B500AF534B32
:100220001A68524B802149020A431A60C0464F4B5C
:100230001A6880239B021340F9D04C4B5A684B4BF1
:100240004B490A405A60494B5A68484B8821490338
:100250000A435A60454B1A68444B802149040A43BB
:100260001A60C046414B1A6880239B041340F9D0A2
:100270003E4B5A683D4B02210A435A6000F072FE21
:100280003C4B1B680A21180001F0EEF9030018002E
:10029000FFF79AFF01235B421800FFF711FF0123CC
:1002A0005B4260211800FFF721FF304B5A692F4B4A
:1002B00031490A435A612D4B9A692C4B2F490A4305
:1002C0009A612A4BDA69294B02210A43DA619023A9
:1002D000DB051A689023DB0529490A431A6090233D
:1002E000DB059A689023DB0526490A439A60902330
:1002F000DB0500221A629023DB05882252005A6235
:10030000214A214B12681A60204BC92292001A60C0
:100310001E4BE022D2005A601C4B1A681B4B402136
:100320000A431A601920FFF7CBFE40211920FFF77E
:10033000DDFE174B00225A60154B0122DA60144B88
:100340002F229A62124B134ADA62114B01221A6071
:100350001520FFF7B5FE40211520FFF7C7FE0E4B15
:10036000180000F045F900F0CDFAFEE70010024059
:100370000CF8C3FF0000002011000600015A4200E3
:1003800070A92800808A080000040048003001405D
:1003900000440140E703000040420F0080B500AF79
:1003A000084B9B680222134009D09023DB050822EA
:1003B0009A61044B5A68034B80218A435A60C046B5
:1003C000BD4680BD0030014080B582B000AF284BF3
:1003D0001B690122134047D0254B1A69244B012188
:1003E0008A431A61FB1D00221A70BB1D01221A707C
:1003F00000233B601DE01F4B3A689200D358002B4E
:100400000FD01C4B3A689200D358591E194B3A68CA
:100410009200D150FB1DF91DBA1D097812780A43CC
:100420001A70BA1DBB1D1B78DB1813703B680133B3
:100430003B603B68072BDED90F4B1B68591C0E4AEB
:1004400011600A2B10D10C4B00221A600B4AFB1DC5
:100450001B7813700A4B5A68094B80210A435A6073
:100460009023DB0508229A62C046BD4602B080BDDB
:1004700000440140B0000020980000200C300140F2
:100480000030014080B500AF00BEC046BD4680BD13
:1004900000BEC04680B500AF00BEC046BD4680BDB0
:1004A00080B500AF00BEC046BD4680BD80B500AF80
:1004B0000A4B1B68591C094A11600A2B0AD1074BC9
:1004C00000221A60064B1B685A1C054B1A60054B2C
:1004D00064229A61C046BD4680BDC0469C00002093
:1004E00094000020B000002080B582B000AF020070
:1004F000FB1D1A70FB1D1B781A001F231A40044BAA
:10050000012191400A001A60C046BD4602B080BD7C
:1005100000E100E090B583B000AF02003960FB1D40
:100520001A70FB1D1B787F2B32D92F4AFB1D1B78BD
:1005300019000F230B40083B9B0806339B00D31880
:1005400004331B68FA1D1278110003220A40D200FE
:10055000FF2191400A00D2431A4011003B689B01E1
:10056000FF221A40FB1D1B78180003230340DB0009
:100570009A401D48FB1D1B781C000F232340083B9D
:100580009B080A4306339B00C31804331A6027E014
:10059000164AFB1D1B785BB29B08C0339B009B581F
:1005A000FA1D1278110003220A40D200FF21914067
:1005B0000A00D2431A4011003B689B01FF221A40F7
:1005C000FB1D1B78180003230340DB009A400748FB
:1005D000FB1D1B785BB29B080A43C0339B001A507B
:1005E000C046BD4603B090BD00ED00E000E100E074
:1005F00080B584B000AF7860202000F04BF8214B2C
:10060000802212061A611F4B07225A611D4B1E4A97
:10061000DA601C4B04229A621A4B9A68194B8021AB
:1006200009060A439A60C046164B9B68002BFBDB09
:10063000144B9A68134B01210A439A60114B9A6834
:10064000104B04210A439A607B68104A934206DDEE
:100650007B68FA21180001F091F8030000E00623FE
:10066000FB60FA6880235B029A4201DB084BFB6067
:10067000FB6819000C2000F03DF8C046BD4604B0F0
:1006800080BDC0460024014043080000DC05000096
:10069000FFFF000080B582B000AF7860114B124AB6
:1006A0009A60104B114ADA600E4B7A685A600D4B13
:1006B00000221A600B4B1A680A4B0D490A431A6054
:1006C0000920FFF711FF60210920FFF723FF054BE9
:1006D0001A68044B01210A431A60C046BD4602B0A5
:1006E00080BDC0460800024040240140D0000020E8
:1006F000A605000080B582B000AF78603960154B68
:10070000802212025A64134BC022D201DA61114BCB
:10071000802252011A620F4B01221A647B685A1E12
:100720000C4B9A623B685A1E0A4BDA62094B5A69B3
:10073000084B01210A435A61064B80221A60054B7F
:100740001A68044B01210A431A60C046BD4602B034
:1007500080BDC046002C014080B500AFC046BD46FC
:1007600080BD80B582B000AF144B1B683B60134B5B
:100770005A68124B01210A435A60FFF7EDFF3B68AC
:100780004022134007D00E4B2021180000F0C6F97C
:1007900003007B6006E00B4B2021180000F0BEF93F
:1007A00003007B607B68002B04D0074B1B685A1C3E
:1007B000054B1A60C046BD4602B080BD0000024035
:1007C000D0000020E0000020A000002080B582B012
:1007D00000AF0200FB1D1A70FB1D1B781A001F23BF
:1007E0001A40044B012191400A001A60C046BD46E0
:1007F00002B080BD00E100E080B582B000AF020031
:10080000FB1D1A70FB1D1B781A001F23134005499E
:1008100001229A40130080228B50C046BD4602B090
:1008200080BDC04600E100E090B583B000AF02009B
:100830003960FB1D1A70FB1D1B787F2B32D92F4AA4
:10084000FB1D1B7819000F230B40083B9B08063348
:100850009B00D31804331B68FA1D12781100032281
:100860000A40D200FF2191400A00D2431A401100F1
:100870003B689B01FF221A40FB1D1B7818000323D5
:100880000340DB009A401D48FB1D1B781C000F2312
:100890002340083B9B080A4306339B00C3180433DC
:1008A0001A6027E0164AFB1D1B785BB29B08C03319
:1008B0009B009B58FA1D1278110003220A40D200B7
:1008C000FF2191400A00D2431A4011003B689B016E
:1008D000FF221A40FB1D1B78180003230340DB0096
:1008E0009A400748FB1D1B785BB29B080A43C03344
:1008F0009B001A50C046BD4603B090BD00ED00E01D
:1009000000E100E080B500AF194B012252421A60AD
:10091000174B00225A60164B00229A60154B164A5C
:100920009A60144B92221A600A20FFF74FFF202191
:100930000A20FFF779FF114B114A1A600F4B602212
:10094000DA600E4BC022DA600C4BC02292025A6071
:100950000A4B9A68094B80210A439A60074B1A6830
:10096000064B01210A431A60C046BD4680BDC04601
:10097000100100201C0002402838014000380140CE
:100980002C20000080B584B000AF194BBB60BB6861
:100990005B687B60BB689B687A689A4205D2BB68DB
:1009A0009A687B68D31AFB6004E07B688022D200DF
:1009B000D31AFB60BB687A681A607A68FB68D31840
:1009C0009B059A0DBB685A60BB680C331A007B68A4
:1009D000D218084BDA60074BFA685A60054B1A6860
:1009E000044B01210A431A60C046BD4604B080BDD5
:1009F000100100201C00024080B582B000AF78607A
:100A00000A00FB1C1A700A20FFF7F6FE7B689A6842
:100A10007B681B689A4205D10A20FFF7D7FE102396
:100A20005B4211E07B689B687A68D318FA1C1278E5
:100A30001A737B689B6801339B059A0D7B689A60EB
:100A40000A20FFF7C3FE00231800BD4602B080BD98
:100A500080B582B000AF0200FB1D1A70C046FB1DBE
:100A60001A78064B11001800FFF7C6FF0300103379
:100A7000F5D000231800BD4602B080BD1001002053
:100A800080B582B000AF0200FB1D1A70FB1D1A7802
:100A9000044B11001800FFF7AFFF03001800BD461C
:100AA00002B080BD1001002080B500AF0B4B5A682A
:100AB0000A4B20210A435A60094B1A68084B01214E
:100AC0008A431A60074B9A68064B5B689A4201D0CA
:100AD000FFF758FFC046BD4680BDC046000002403B
:100AE0001C0002401001002080B582B000AF786089
:100AF00039603A687968074B180000F09CF8064B9B
:100B00001B680122134001D1FFF73CFFC046BD46E0
:100B100002B080BD510A00081C00024080B584B0BC
:100B200000AF786039600023FB600BE00E4B1B7850
:100B30005A1CD1B20C4A11701800FFF7A1FFFB68D4
:100B40000133FB60FA68AF235B009A42EED9074B92
:100B50001B680122134001D1FFF714FF0023180086
:100B6000BD4604B080BDC046A40000201C00024069
:100B700080B588B000AFF860B9607A603B60BA6851
:100B800080235B029A4202D23B68FE2B02D90123EA
:100B90005B424CE03B680233BA689A4202D20123BE
:100BA0005B4244E00023FB6136E0FB69002B0FD081
:100BB000FB69013B7A68D3181B78002B08D0FB69CE
:100BC000013B7A68D2181B23FB1812781A7019E0BF
:100BD000FB697B6102E07B6901337B617A693B6879
:100BE0009A4205D27A687B69D3181B78002BF2D120
:100BF0007B69DAB2FB69DBB2D31ADAB21B23FB18CA
:100C000001321A70FA68FB69D3181B22BA181278DD
:100C10001A70FB690133FB61FA693B689A42C4D9D7
:100C2000FA68FB69D31800221A703B680233180077
:100C3000BD4608B080BD80B58AB000AFF860B9602D
:100C40007A607B68FE2B02D901235B424EE00023D1
:100C50007B623CE07B6A002B0FD07B6A013BBA6869
:100C6000D3181B78002B08D07B6A013BBA68D218D6
:100C70002323FB1812781A7019E07B6AFB6102E0EB
:100C8000FB690133FB61FA697B689A4205D2BA6855
:100C9000FB69D3181B78002BF2D1FB69DAB27B6AAF
:100CA000DBB2D31ADAB22323FB1801321A702323E2
:100CB000FB181A78FB681000984703007B617B697A
:100CC000002B01D07B6911E07B6A01337B627A6A79
:100CD0007B689A42BED9FB68002098470300BB613D
:100CE000BB69002B01D0BB6900E000231800BD46A2
:100CF0000AB080BD80B588B000AFF860B9607A6096
:100D00003B60BA6880235B029A4204D23A6880232F
:100D10005B029A4202D301235B4252E03B68002B04
:100D200002D101235B424CE0BA683B689A4202D28E
:100D300001235B4245E00123FB617B681B78BB61BB
:100D4000BB69002B24D102235B423AE0BB69013B23
:100D5000BB61BB69002B09D17A68FB69D3181B788A
:100D6000BB611723FB1800221A7006E07A68FB6942
:100D7000D2181723FB1812781A70FB69013BFA6826
:100D8000D3181722BA1812781A70FB690133FB6165
:100D9000FA693B689A4205D27A68FB69D3181B78D6
:100DA000002BD3D1FA693B689A4202D102235B42FD
:100DB00007E0BB69012B02D003235B4201E0FB6922
:100DC000013B1800BD4608B080BD80B582B000AFC1
:100DD00078607B6800221A607B6800225A60C046F7
:100DE000BD4602B080BD80B588B000AFF860B96084
:100DF0007A601A00FB1C1A70FB681B68002B0ED16E
:100E0000FB1C1B78002B54D0FB1C1A78FB685A6023
:100E1000FB681B685A1CFB681A60002350E0FB1C2F
:100E20001B78002B0DD1FB685B68012B39D1FB6867
:100E30001B68013B7B61FB681800FFF7C6FF7B69FD
:100E40003EE0FB685B685A1EFB685A60FB685B68A3
:100E5000002B08D1FB1C1A78FB685A601F23FB1873
:100E600000221A7004E01F23FB18FA1C12781A7073
:100E7000FB681B68013BBB61BA697B689A4202D37D
:100E800002235B421CE0BA68BB69D3181F22BA1860
:100E900012781A70FB681B685A1CFB681A600023E2
:100EA0000EE0C046FB681800FFF78FFF01235B428E
:100EB00006E0C046FB681800FFF787FF03235B428C
:100EC0001800BD4608B080BDBC1900080000002015
:100ED00094000020940000201C05002080B500AF85
:100EE0001A4B1A68194B01210A431A60174B5A68AA
:100EF000164B17490A405A60144B1A68134B154990
:100F00000A401A60114B1A68104B13490A401A60C4
:100F10000E4B5A680D4B11490A405A600B4BDA6A66
:100F20000A4B0F218A43DA62084B1A6B074B0C49B4
:100F30000A401A63054B5A6B044B01218A435A63DA
:100F4000024B00229A60C046BD4680BD00100240A0
:100F50000CB8FF08FFFFF6FEFFFFFBFFFFFFC0FF1F
:100F6000ECFEFFFF80B584B000AF0023FB600023E0
:100F7000BB6000237B6000233B60314B5B680C222D
:100F80001340FB60FB68082B11D0FB68082B41D88D
:100F9000FB68002B03D0FB68042B04D03AE0294BFC
:100FA000294A1A603AE0274B274A1A6036E0244B58
:100FB0005A68F0239B031340BB60214B5A6880237F
:100FC0005B0213407B60BB689B0C0233BB601C4B15
:100FD000DB6A0F22134001333B607A6880235B0297
:100FE0009A420AD13968184800F03EFB03001A0003
:100FF000BB685A43134B1A6010E0B9680A005201EB
:10100000521A93019B1ADB005B181B021A000D4B4E
:101010001A6003E00B4B0C4A1A60C046084B5B6831
:101020001B090F221340094AD35CFB60054B1A6869
:10103000FB68DA40034B1A60C046BD4604B080BD71
:10104000001002400000002000127A00A4190008DD
:1010500080B500AF044B1A68034B8021C9020A43D4
:101060001A60C046BD4680BD0010024080B500AF8A
:10107000044B1A68034B04490A401A60C046BD4637
:1010800080BDC04600100240FFFFFBFF80B500AFEF
:10109000044B1A68034B802149020A431A60C04678
:1010A000BD4680BD0010024080B500AF064B1A68F7
:1010B00080239B021340054A944663445A4253419D
:1010C000DBB21800BD4680BD001002400000FEFFEC
:1010D00080B500AF044B1A68034B01210A431A6024
:1010E000C046BD4680BDC0460010024080B500AF7E
:1010F000054B1B6802221340023B5A425341DBB2AC
:101100001800BD4680BDC0460010024080B582B0C8
:1011100000AF7860064B5B68032293431900044BD1
:101120007A680A435A60C046BD4602B080BDC046D8
:101130000010024080B500AF034B5B680C221340E7
:101140001800BD4680BDC0460010024080B582B088
:1011500000AF7860064B5B68F02293431900044BA4
:101160007A680A435A60C046BD4602B080BDC04698
:101170000010024080B582B000AF7860064B5B681B
:10118000064A13401900044B7A680A435A60C04665
:10119000BD4602B080BDC04600100240FFF8FFFF10
:1011A00080B500AF044B1A68034B802149040A4301
:1011B0001A60C046BD4680BD0010024080B500AF39
:1011C000074B1A6880239B041340FE2212069446A4
:1011D00063445A425341DBB21800BD4680BDC0464D
:1011E0000010024080B582B000AF786039600E4BCD
:1011F0005B680E4A134019007A6880235B021A402C
:101200003B681A43084B0A435A60074BDB6A0F22BC
:10121000934319007B680F221A40034B0A43DA629A
:10122000C046BD4602B080BD00100240FFFFC2FFB5
:1012300080B582B000AF786039603968786800F0B6
:1012400013FA03001A00064B013A5A60044B0022BD
:101250009A60034B05221A60C046BD4602B080BDAD
:1012600010E000E080B582B000AF7860064B1B68EC
:10127000012293431900044B7A680A431A60C0465E
:10128000BD4602B080BDC0460020024080B500AF20
:10129000034B1B68012213401800BD4680BDC046A9
:1012A0000020024080B582B000AF7860FA239A0037
:1012B0007B6811001800FFF7BBFFC046BD4602B0B7
:1012C00080BD80B584B000AF78600E4B1B68FB60BA
:1012D000FB687B6801330CD07B6801337B6008E0DE
:1012E000084B1A6880235B02134002D07B68013BE5
:1012F0007B607B68002BF3D1C046C046BD4604B07E
:1013000080BDC04610E000E080B582B000AF7860DC
:10131000034B7A681A60C046BD4602B080BDC04625
:101320000000002090B585B000AF786039600F23D1
:10133000FB1801221A700023BB6000F0D4F80300F0
:10134000012B28D17B6801225A607B68174A19005B
:10135000100000F0ABF80300BB60FFF7C7FE03000E
:10136000012B07D0FFF7B4FEC046FFF7BFFE030016
:10137000012BFAD17B681B6819000020FFF732FFB0
:101380000F23FC183A68BB681100180000F0BEF883
:101390000300237003E00F23FB1800221A700F23B1
:1013A000FB181B781800BD4605B090BD00127A00EE
:1013B00090B587B000AFF860B9607A603B601723E2
:1013C000FB1801221A7000233B6100F08CF8030027
:1013D000012B32D17A68FB681100180000F066F822
:1013E00003003B61FFF760FE0300012B0FD0BB68D9
:1013F000012B02D1FFF72CFE01E0FFF737FEFFF7CC
:1014000045FEC046FFF750FE0300012BFAD17B6872
:101410005B68802252021A437B681B681900100027
:10142000FFF7E0FE1723FC183A683B69110018002B
:1014300000F06CF80300237003E01723FB18002270
:101440001A701723FB181B781800BD4607B090BD13
:1014500080B584B000AF78600F217B1801221A702C
:101460000023BB607B68002B03D17B1800221A701D
:1014700013E07B680C4A934201D90123BB60BB682F
:101480001800FFF7EFFEFFF701FF0200BB68934271
:1014900003D00F23FB1800221A700F23FB181B78B0
:1014A0001800BD4604B080BD00366E0180B584B022
:1014B00000AF786039600023FB603B685B680133F4
:1014C0001900786800F0D0F8030019003B681B6829
:1014D0009B0C0F22134002334B43FB60FB68180048
:1014E000BD4604B080BD80B582B000AFFB1D0122B7
:1014F0001A70FFF763FE031E02D0FB1D00221A7054
:10150000FB1D1B781800BD4602B080BD90B585B0AC
:1015100000AF786039600F203B1801221A70002359
:10152000BB602E4B1A683B681B681B090F210B40E0
:101530002B49CB5C9A401300BB60BA687B689A4227
:1015400006D23C187B681800FFF782FF0300237067
:101550000F23FB181B78012B1AD1FFF721FEC04681
:10156000FFF72CFE0300012BFAD13B681B68180023
:10157000FFF7ECFD0220FFF7C9FDC046FFF7DAFDDB
:101580000300082BFAD13B685B681800FFF7F2FDF7
:10159000BA687B689A4207D90F23FC187B68180049
:1015A000FFF756FF030023700F23FB181B78012B56
:1015B0000CD13B681B681B090F221340084AD35CFF
:1015C0001A007B68D3401800FFF79EFE0F23FB181C
:1015D0001B781800BD4605B090BDC0460000002035
:1015E000A419000880B500AFC046BD4680BD80B5D7
:1015F00086B000AFF860B9607A60FA687B68D3188B
:101600003B61FB687B6106E0BB68DAB27B691A70FC
:101610007B6901337B617A693B699A42F4D3FB6849
:101620001800BD4606B080BD80B584B000AF7860BC
:101630007B68FB60C0467B685A1C7A601B78002B75
:10164000F9D17A68FB68D31A013B1800BD4604B093
:1016500080BD80B582B000AF0200FB1D1A70C0468D
:10166000BD4602B080BD0000002243088B4274D307
:1016700003098B425FD3030A8B4244D3030B8B4293
:1016800028D3030C8B420DD3FF22090212BA030C9C
:101690008B4202D31212090265D0030B8B4219D37D
:1016A00000E0090AC30B8B4201D3CB03C01A52419D
:1016B000830B8B4201D38B03C01A5241430B8B42E5
:1016C00001D34B03C01A5241030B8B4201D30B03CE
:1016D000C01A5241C30A8B4201D3CB02C01A5241F5
:1016E000830A8B4201D38B02C01A5241430A8B42B8
:1016F00001D34B02C01A5241030A8B4201D30B02A1
:10170000C01A5241CDD2C3098B4201D3CB01C01ABA
:10171000524183098B4201D38B01C01A52414309C4
:101720008B4201D34B01C01A524103098B4201D3B2
:101730000B01C01A5241C3088B4201D3CB00C01A1F
:10174000524183088B4201D38B00C01A5241430897
:101750008B4201D34B00C01A5241411A00D20146BC
:10176000524110467047FFE701B5002000F0F0F845
:1017700002BDC0460029F7D076E7704703460B4309
:101780007FD4002243088B4274D303098B425FD37A
:10179000030A8B4244D3030B8B4228D3030C8B42A6
:1017A0000DD3FF22090212BA030C8B4202D312128C
:1017B000090265D0030B8B4219D300E0090AC30B61
:1017C0008B4201D3CB03C01A5241830B8B4201D30E
:1017D0008B03C01A5241430B8B4201D34B03C01AF7
:1017E0005241030B8B4201D30B03C01A5241C30A6F
:1017F0008B4201D3CB02C01A5241830A8B4201D3E0
:101800008B02C01A5241430A8B4201D34B02C01AC9
:101810005241030A8B4201D30B02C01A5241CDD26E
:10182000C3098B4201D3CB01C01A524183098B42B9
:1018300001D38B01C01A524143098B4201D34B01A2
:10184000C01A524103098B4201D30B01C01A524105
:10185000C3088B4201D3CB00C01A524183088B428C
:1018600001D38B00C01A524143088B4201D34B0075
:10187000C01A5241411A00D20146524110467047E7
:101880005DE0CA0F00D04942031000D340425340EC
:1018900000229C4603098B422DD3030A8B4212D3AC
:1018A000FC22890112BA030A8B420CD389019211DE
:1018B0008B4208D3890192118B4204D389013AD01B
:1018C000921100E08909C3098B4201D3CB01C01AF0
:1018D000524183098B4201D38B01C01A5241430903
:1018E0008B4201D34B01C01A524103098B4201D3F1
:1018F0000B01C01A5241C3088B4201D3CB00C01A5E
:10190000524183088B4201D38B00C01A5241D9D275
:1019100043088B4201D34B00C01A5241411A00D2F6
:101920000146634652415B10104601D34042002BF2
:1019300000D54942704763465B1000D3404201B571
:10194000002000F005F802BD0029F8D016E7704726
:101950007047C0460C488546002103E00B4B5B589E
:10196000435004310A480B4B42189A42F6D30A4AB4
:1019700002E0002313600432084B9A42F9D3FFF7C8
:10198000ADFAFEF74AFCFEE700100020BC19000883
:101990000000002094000020940000201C0500207E
:1019A000FEE7000000000000000000000102030448
:0C19B00006070809000000000102030403
:1019BC0000127A0000040040002000400028004083
:1019CC00002C0040003000400054004000700040EB
:1019DC0000000140000401400024014008270140A0
:1019EC0008270140002C0140003001400038014024
:1019FC0000440140004801400058014000000240F2
:101A0C00080002401C00024030000240440002402A
:101A1C00580002400020024000F8FF1F0010024056
:101A2C000030024000000048000400480008004854
:101A3C00000C00480014004800ED00E010E000E04D
:041A4C0000E100E0D5
:040000050800195581
:00000001FF
